:020000040000fa
:080000000002040000000000f2
:020000040000fa
:040008005e04000092
:020000040000fa
:04000c00ac03000041
:020000040000fa
:04001000ee030000fb
:020000040000fa
:04001400cc03000019
:020000040000fa
:040018000e040000d2
:020000040000fa
:04001c005e0400007e
:020000040000fa
:040020005e0400007a
:020000040000fa
:040024005e04000076
:020000040000fa
:040028005e04000072
:020000040000fa
:04002c005e0400006e
:020000040000fa
:040030005e0400006a
:020000040000fa
:040034002e04000096
:020000040000fa
:040038005e04000062
:020000040000fa
:04003c005e0400005e
:020000040000fa
:040040005e0400005a
:020000040000fa
:040044005e04000056
:020000040000fa
:040048005e04000052
:020000040000fa
:04004c005e0400004e
:020000040000fa
:040050005e0400004a
:020000040000fa
:040054005e04000046
:020000040000fa
:040058005e04000042
:020000040000fa
:04005c005e0400003e
:020000040000fa
:040060005e0400003a
:020000040000fa
:040064005e04000036
:020000040000fa
:040068005e04000032
:020000040000fa
:04006c005e0400002e
:020000040000fa
:040070005e0400002a
:020000040000fa
:040074005e04000026
:020000040000fa
:040078005e04000022
:020000040000fa
:04007c005e0400001e
:020000040000fa
:040080005e0400001a
:020000040000fa
:040084005e04000016
:020000040000fa
:040088005e04000012
:020000040000fa
:04008c005e0400000e
:020000040000fa
:040090005e0400000a
:020000040000fa
:040094005e04000006
:020000040000fa
:040098005e04000002
:020000040000fa
:04009c005e040000fe
:020000040000fa
:0400a0005e040000fa
:020000040000fa
:0400a4005e040000f6
:020000040000fa
:0400a8005e040000f2
:020000040000fa
:0400ac005e040000ee
:020000040000fa
:0400b0005e040000ea
:020000040000fa
:0400b4005e040000e6
:020000040000fa
:0400b8005e040000e2
:020000040000fa
:0400bc005e040000de
:020000040000fa
:0400c0005e040000da
:020000040000fa
:0400c4005e040000d6
:020000040000fa
:0400c8005e040000d2
:020000040000fa
:0400cc005e040000ce
:020000040000fa
:0400d0005e040000ca
:020000040000fa
:0400d4005e040000c6
:020000040000fa
:0400d8005e040000c2
:020000040000fa
:0400dc005e040000be
:020000040000fa
:0400e0005e040000ba
:020000040000fa
:0400e4005e040000b6
:020000040000fa
:0400e8005e040000b2
:020000040000fa
:0400ec00cc02000042
:020000040000fa
:0400f0005e040000aa
:020000040000fa
:0400f4005e040000a6
:020000040000fa
:0400f8005e040000a2
:020000040000fa
:0400fc005e0400009e
:020000040000fa
:040100005e04000099
:020000040000fa
:040104005e04000095
:020000040000fa
:040108005e04000091
:020000040000fa
:04010c005e0400008d
:020000040000fa
:040110005e04000089
:020000040000fa
:040114005e04000085
:020000040000fa
:040118005e04000081
:020000040000fa
:04011c005e0400007d
:020000040000fa
:040120005e04000079
:020000040000fa
:040124005e04000075
:020000040000fa
:040128005e04000071
:020000040000fa
:04012c005e0400006d
:020000040000fa
:040130005e04000069
:020000040000fa
:040134005e04000065
:020000040000fa
:040138005e04000061
:020000040000fa
:04013c005e0400005d
:020000040000fa
:040140005e04000059
:020000040000fa
:040144005e04000055
:020000040000fa
:040148005e04000051
:020000040000fa
:04014c005e0400004d
:020000040000fa
:040150005e04000049
:020000040000fa
:040154005e04000045
:020000040000fa
:040158005e04000041
:020000040000fa
:04015c005e0400003d
:020000040000fa
:040160005e04000039
:020000040000fa
:040164005e04000035
:020000040000fa
:040168005e04000031
:020000040000fa
:04016c005e0400002d
:020000040000fa
:040170005e04000029
:020000040000fa
:040174005e04000025
:020000040000fa
:040178005e04000021
:020000040000fa
:04017c005e0400001d
:020000040000fa
:040180005e04000019
:020000040000fa
:040184005e04000015
:020000040000fa
:040188005e04000011
:020000040000fa
:04018c005e0400000d
:020000040000fa
:040190005e04000009
:020000040000fa
:040194005e04000005
:020000040000fa
:040198005e04000001
:020000040000fa
:04019c005e040000fd
:020000040000fa
:0401a0005e040000f9
:020000040000fa
:0401a4005e040000f5
:020000040000fa
:0401a8005e040000f1
:020000040000fa
:0401ac005e040000ed
:020000040000fa
:040208005e04000090
:020000040000fa
:04020c00ac0300003f
:020000040000fa
:04021000ee030000f9
:020000040000fa
:04021400cc03000017
:020000040000fa
:040218000e040000d0
:020000040000fa
:04021c005e0400007c
:020000040000fa
:040220005e04000078
:020000040000fa
:040224005e04000074
:020000040000fa
:040228005e04000070
:020000040000fa
:04022c005e0400006c
:020000040000fa
:040230005e04000068
:020000040000fa
:040234002e04000094
:020000040000fa
:040238005e04000060
:020000040000fa
:04023c005e0400005c
:020000040000fa
:040240005e04000058
:020000040000fa
:040244005e04000054
:020000040000fa
:040248005e04000050
:020000040000fa
:04024c005e0400004c
:020000040000fa
:040250005e04000048
:020000040000fa
:040254005e04000044
:020000040000fa
:040258005e04000040
:020000040000fa
:04025c005e0400003c
:020000040000fa
:040260005e04000038
:020000040000fa
:040264005e04000034
:020000040000fa
:040268005e04000030
:020000040000fa
:04026c005e0400002c
:020000040000fa
:040270005e04000028
:020000040000fa
:040274005e04000024
:020000040000fa
:040278005e04000020
:020000040000fa
:04027c005e0400001c
:020000040000fa
:040280005e04000018
:020000040000fa
:040284005e04000014
:020000040000fa
:040288005e04000010
:020000040000fa
:04028c005e0400000c
:020000040000fa
:040290005e04000008
:020000040000fa
:040294005e04000004
:020000040000fa
:040298005e04000000
:020000040000fa
:04029c005e040000fc
:020000040000fa
:0402a0005e040000f8
:020000040000fa
:0402a4005e040000f4
:020000040000fa
:0402a8005e040000f0
:020000040000fa
:0402ac005e040000ec
:020000040000fa
:0402b0005e040000e8
:020000040000fa
:0402b4005e040000e4
:020000040000fa
:0402b8005e040000e0
:020000040000fa
:0402bc005e040000dc
:020000040000fa
:0402c0005e040000d8
:020000040000fa
:0402c4005e040000d4
:020000040000fa
:0402c8005e040000d0
:020000040000fa
:0402cc005e040000cc
:020000040000fa
:0402d0005e040000c8
:020000040000fa
:0402d4005e040000c4
:020000040000fa
:0402d8005e040000c0
:020000040000fa
:0402dc005e040000bc
:020000040000fa
:0402e0005e040000b8
:020000040000fa
:0402e4005e040000b4
:020000040000fa
:0402e8005e040000b0
:020000040000fa
:0402ec00cc02000040
:020000040000fa
:0402f0005e040000a8
:020000040000fa
:0402f4005e040000a4
:020000040000fa
:0402f8005e040000a0
:020000040000fa
:0402fc005e0400009c
:020000040000fa
:040300005e04000097
:020000040000fa
:040304005e04000093
:020000040000fa
:040308005e0400008f
:020000040000fa
:04030c005e0400008b
:020000040000fa
:040310005e04000087
:020000040000fa
:040314005e04000083
:020000040000fa
:040318005e0400007f
:020000040000fa
:04031c005e0400007b
:020000040000fa
:040320005e04000077
:020000040000fa
:040324005e04000073
:020000040000fa
:040328005e0400006f
:020000040000fa
:04032c005e0400006b
:020000040000fa
:040330005e04000067
:020000040000fa
:040334005e04000063
:020000040000fa
:040338005e0400005f
:020000040000fa
:04033c005e0400005b
:020000040000fa
:040340005e04000057
:020000040000fa
:040344005e04000053
:020000040000fa
:040348005e0400004f
:020000040000fa
:04034c005e0400004b
:020000040000fa
:040350005e04000047
:020000040000fa
:040354005e04000043
:020000040000fa
:040358005e0400003f
:020000040000fa
:04035c005e0400003b
:020000040000fa
:040360005e04000037
:020000040000fa
:040364005e04000033
:020000040000fa
:040368005e0400002f
:020000040000fa
:04036c005e0400002b
:020000040000fa
:040370005e04000027
:020000040000fa
:040374005e04000023
:020000040000fa
:040378005e0400001f
:020000040000fa
:04037c005e0400001b
:020000040000fa
:040380005e04000017
:020000040000fa
:040384005e04000013
:020000040000fa
:040388005e0400000f
:020000040000fa
:04038c005e0400000b
:020000040000fa
:040390005e04000007
:020000040000fa
:040394005e04000003
:020000040000fa
:040398005e040000ff
:020000040000fa
:04039c005e040000fb
:020000040000fa
:0403a0005e040000f7
:020000040000fa
:0403a4005e040000f3
:020000040000fa
:0403a8005e040000ef
:020000040000fa
:0403ac005e040000eb
:020000040000fa
:10040000cf8520000eff20000e01880000000000b4
:10041000000020000000e000020032000001200087
:100420002002880014000700260107000000e000f9
:1004300003003a0060b420000100200002003700f1
:100440000000200001002000810f70000100320038
:1004500014000700000020000000e000020032004d
:100460000000020000000000be0a020000000000c0
:100470000040da000000fe004440a9000000200017
:100480000000e0000300320000002000a00188000e
:100490004440a800000006008a1f78008b1f7800e7
:1004a0000000060091018800800478000000eb0045
:1004b0001a003700e284440032a0b4009905ba0063
:1004c000e284440032a0b4009906ba00e2844400f9
:1004d00032a0b4000006eb00476fde00fd07b2005b
:1004e000636ce10003003a00ebff07000000eb0043
:1004f0000a003700606ce10004003a00005deb0088
:100500008b05e900fdff3e00040037006168e10053
:10051000010032000086eb000b00070019c7ba008b
:100520001905ba000e04e00003003a000a00e000da
:10053000e0ff3a0000000600fe07b2009e018800be
:100540008a047800f5ff3700395dba008b05e900b1
:100550000c003200295dba008b05e900080032006a
:100560000c00e00003003a00e284440032a0b40032
:10057000f5ff370019ddba008b05e900faff3a00f4
:100580008904e800e184440032a0b40000000600c1
:100590000000000000000000809fbe00821f780065
:1005a0000000fa0050048000620060000000e000db
:1005b00046003200c0108000640060000000e000cf
:1005c00007003200801080000040780040e8b7004b
:1005d00042c8bf000080fb00801088001282a80083
:1005e000c0108000640060000000e00037003a00a6
:1005f0000021ef00c1108000000220000080600098
:100600000000e00015003a0061168000000820009c
:100610000080600000f0a7000000ea000000e90090
:100620004f00de00004078000080fb0061006000a9
:100630004700dd00611680000170a100010070001c
:100640006016880010c0b3004be8b700801080002f
:100650000040780040e8b7001282a800c110800076
:1006600000022000008060000000e000170032005f
:100670004bc8bf00e14f500005003a0080108000d9
:10068000004078003fe8b7004b68ef000e003700ed
:100690003fc8bf00e54f500008003e003fc8bf0004
:1006a0000081fb00801080008040780010842000d2
:1006b00000004100014878000300370080108000ee
:1006c0000040780040e8b7001282a8005004800083
:1006d000640060000000e00005003a009110800016
:1006e00000042000008060000000e00006003200ee
:1006f000801080000040780040e8b7008a40a900e0
:1007000012c2a9001282a8008a20a90091108000bc
:10071000000420000080600000f0a7000000ea0054
:100720000000e9004f00de00004078000080fb0080
:10073000610060004800dd00611680000180a100ba
:1007400001007000601688000080fa004f017800f8
:100750004f00be00004006003600f800809fbe003b
:10076000829fbe00849fbe00869fbe000000fa00ec
:100770008020a9000000eb00ff0307000080fa00c2
:100780004f03be004f02be004f01be004f00be002f
:100790003600f900004006003600f800809fbe00d9
:1007a000829fbe00849fbe00869fbe000000fa00ac
:1007b000f60307008040a90010002000ee030700a8
:1007c0000080fa004f03be004f02be004f01be0082
:1007d0004f00be003600f900004006003600f80069
:1007e000809fbe00829fbe00849fbe00869fbe0089
:1007f0000000fa008060a90020002000de0307004e
:100800000080fa004f03be004f02be004f01be0041
:100810004f00be003600f900004006003600f80028
:10082000809fbe00829fbe00849fbe00869fbe0048
:100830000000fa008080a90030002000ce030700ed
:100840000080fa004f03be004f02be004f01be0001
:100850004f00be003600f900004006003600f800e8
:10086000809fbe00829fbe00849fbe00869fbe0008
:100870000000fa00a04280000000e0000200320008
:10088000a04280000000010057c8bf000040e800ff
:1008900057e8b70010c0b30056e8b7008460a9005d
:1008a0000080fa004f03be004f02be004f01be00a1
:1008b0004f00be003600f900004006000040da009c
:0808c0000000fe00000005002d
:020000040000fa
:1008c8000400fa00004f780011479800224798006a
:1008d8001e407800ef4f500002003600f0c0b30011
:1008e800004f78001e409000e54f5000020036008f
:1008f80050c0b3001047980000c8b30024e8b70000
:1009080024c8bf0022e8b70022c8bf0020e8b7000b
:100918001e80fb00f10f20000008dd0000f0a7009a
:100928000000ea000000e9004f00de000040780007
:1009380025e8b7001e80fb0068005000f10f20007a
:100948000008dd0000f0a7000000ea000000e90050
:100958004f00de00804078001e4090000080fb00c1
:10096800640050004700dd000040780000c07000bf
:1009780023e8b7001e4090000080fb000000e9005b
:10098800f10f20000008dd0000f0a7000000ea00d9
:100998000000e9004f00de00804078002e40900003
:1009a8000080fb004700dd000040780000c07000b8
:1009b80021e8b7006282200061c0b30000822000f5
:1009c800cb0107000080fb00704188000080fa001e
:1009d800000006000200fa00000f780032c8bf00cd
:1009e8000080fb004800dd008040780032c8bf006e
:1009f8000004e00002003a0000c8b300010037001c
:100a08000040eb0000c070000004a00024e8b7001c
:100a180024c8bf0022e8b70022c8bf0020e8b700fa
:100a28001e0078001040780021e8b7001e00e8009a
:100a38001040780023e8b7001e80e80010407800d6
:100a480025e8b7000080fa00000006000200fa005e
:100a5800000f780032c8bf000080fb004800dd00ae
:100a68008040780032c8bf000004e00002003a006d
:100a780000c8b300010037000040eb0000c0700060
:100a88000024a00024e8b70024c8bf0022e8b7006b
:100a980022c8bf0020e8b7001e0078001040780088
:100aa80021e8b7001e00e8001040780023e8b700ee
:100ab8001e80e8001040780025e8b7000080fa00a2
:100ac800000006000200fa00000f780032c8bf00dc
:100ad8000080fb004800dd008040780032c8bf007d
:100ae8000004e00002003a0000c8b300010037002b
:100af8000040eb0000c070005040b30024e8b7008d
:100b080024c8bf0022e8b70022c8bf0020e8b70009
:100b18001e0078001040780021e8b7001e00e800a9
:100b28001040780023e8b7001e80e80010407800e5
:100b380025e8b7000080fa00000006000000fa006f
:100b480060c4b30024e8b70024c8bf0022e8b70097
:100b580022c8bf0020e8b7000080fa0000000600a5
:100b68000200fa00000f780032c8bf000080fb00c6
:100b78004800dd008040780032c8bf000004e00073
:100b880002003a0000c8b300010037000040eb0043
:100b980000c070000034a00024e8b70024c8bf00db
:100ba80022e8b70022c8bf0020e8b7001e0078007e
:100bb8001040780021e8b7001e00e80010407800d7
:100bc80023e8b7001e80e8001040780025e8b70049
:100bd8000080fa00000006000000fa0090c4b3008c
:100be80024e8b70024c8bf0022e8b70022c8bf0025
:100bf80020e8b7000080fa00000006000000fa00b4
:100c0800a0c4b30024e8b70024c8bf0022e8b70096
:100c180022c8bf0020e8b7000080fa0000000600e4
:100c28000200fa00000f780032c8bf000080fb0005
:100c38004800dd008040780032c8bf000004e000b2
:100c480002003a0000c8b300010037000040eb0082
:100c580000c07000b040b30024e8b70024c8bf004b
:100c680022e8b70022c8bf0020e8b7001e007800bd
:100c78001040780021e8b7001e00e8001040780016
:100c880023e8b7001e80e8001040780025e8b70088
:100c98000080fa00000006000200fa00000f780049
:100ca800c0c8b30020e8b70000c8b30021e8b70007
:100cb80026c8bf000080fb008000780020c8bf0065
:100cc8000080fb000101780021c0b3000801070083
:100cd8000080fb00704188000080fa0000000600d8
:100ce8000200fa00000f7800d0c8b30024e8b7006b
:100cf80024c8bf0022e8b70022c8bf0020e8b70018
:100d08001e0078001040780021e8b7001e00e800b7
:100d18001040780023e8b7001e80e80010407800f3
:100d280025e8b7000080fa00000006000200fa007b
:100d3800000f780032c8bf000080fb004800dd00cb
:100d48008040780032c8bf000004e00002003a008a
:100d580000c8b300010037000040eb0000c070007d
:100d6800e040b30024e8b70024c8bf0022e8b70079
:100d780022c8bf0020e8b7001e00780010407800a5
:100d880021e8b7001e00e8001040780023e8b7000b
:100d98001e80e8001040780025e8b7000080fa00bf
:100da800000006000200fa00000f780032c8bf00f9
:100db8000080fb004800dd008040780032c8bf009a
:100dc8000004e00002003a0000c8b3000100370048
:100dd8000040eb0000c070000044a00024e8b70009
:100de80024c8bf0022e8b70022c8bf0020e8b70027
:100df80001822000914078001e00780010007800e1
:100e08004600dd004e00de000040780000c07000a3
:100e180020e8b70021822000914078001e80e80079
:100e2800100078004600dd004e00de00004078002b
:100e380000c0700022e8b70041822000914078008d
:100e48001e01780066004100100078004600dd00b1
:100e58004e00de000040780000c0700024e8b700b3
:100e68001e007800100078000040780021e8b700e4
:100e78001e80e800100078000040780023e8b700e2
:100e88009e007800648040001000780000407800e0
:100e980025e8b7000080fa00000006000200fa000a
:100ea800000f780032c8bf000080fb004800dd005a
:100eb8008040780032c8bf000004e00002003a0019
:100ec80000c8b300010037000040eb0000c070000c
:100ed8004041b30024e8b70024c8bf0022e8b700a7
:100ee80022c8bf0020e8b7000182200091407800a6
:100ef8001e007800100078004600dd004e00de007d
:100f08000040780000c0700020e8b700218220006f
:100f1800914078001e80e800100078004600dd004f
:100f28004e00de000040780000c0700022e8b700e4
:100f380041822000914078001e017800660041003f
:100f4800100078004600dd004e00de00004078000a
:100f580000c0700024e8b7001e0078001000780078
:100f68000040780021e8b7001e80e80010007800f3
:100f78000040780023e8b7009e00780064804000b5
:100f8800100078000040780025e8b7000080fa00db
:100f9800000006000200fa00000f780032c8bf0007
:100fa8000080fb004800dd008040780032c8bf00a8
:100fb8000004e00002003a0000c8b3000100370056
:100fc8000040eb0080c0700040c2b30000c0700059
:100fd80024e8b70024c8bf0022e8b70022c8bf0031
:100fe80020e8b7001e0078001040780021e8b7001c
:100ff8001e00e8001040780023e8b7001e80e800d3
:101008001040780025e8b7000080fa0000000600cc
:101018000200fa00000f780032c8bf000080fb0011
:101028004800dd008040780032c8bf000004e000be
:1010380002003a0000c8b300010037000040eb008e
:1010480080c0700050c2b30000c0700024e8b70030
:1010580024c8bf0022e8b70022c8bf0020e8b700b4
:101068001e0078001040780021e8b7001e00e80054
:101078001040780023e8b7001e80e8001040780090
:1010880025e8b7000080fa00000006000000fa001a
:101098000008200040108800a002200010108800de
:1010a8000422ef000622ef000c22ef0010002000bf
:1010b800501088000080fa00000006000200fa00c4
:1010c800004f78001e80fb00001088000000000020
:1010d80040108000610060000000e000fcff32006a
:1010e80000108000004078000080fa000000060030
:1010f8000800fa00881f78001007980041479800f8
:10110800320798000000eb00000f78001e009000e6
:101118000000e0001d0032003e0090000000e000ea
:1011280014003200080037003e0090001e04400002
:101138001e0090001e00400010407800dfff0700ee
:10114800004c78001e0fe8004e4090000080fb0025
:101158009e0f5000f4ff3e001a0037001e0090005a
:101168001e00400010407800d4ff07001e0fe80062
:1011780001003700000000004e4090000080fb0096
:101188009e0f5000f5ff3e000e0037003e00900015
:101198000000e0000b003200060037003e0090001f
:1011a8001e0440000040eb00c4ff0700004c78001c
:1011b8001e0fe8004e4090000080fb009e0f50007c
:1011c800f6ff3e001e007800004078004f047800cb
:1011d8000080fa00000006000000fa0040108000bd
:1011e8006100600000f0a7000000ea000000e900cc
:1011f8004f00de00004078000080fa000000060082
:101208000000fa0011108000000820000080600033
:1012180000f0a7000000ea000000e9004f00de002f
:10122800004078000080fa00000006000000fa0084
:1012380011108000000420000080600000f0a7006a
:101248000000ea000000e9004f00de0000407800de
:101258000080fa00000006000000fa00cde2a900b4
:101268000080fa00000006000000fa00cde2a800a5
:101278000080fa00000006000000fa003628ef009f
:101288000000eb00120007000000eb00160007004a
:1012980000082000c010880060022000901088001c
:1012a80010002000a010880090012000b0108800d5
:1012b8001c22ef0000032000d01088008a40a900fb
:1012c8008a20a9009a20a8000080fa0000000600e1
:1012d8000200fa00000f78009e007800d1418800d3
:1012e8000080fa00000006000200fa00000f7800f3
:1012f8009e007800c14188000080fa0000000600c6
:101308000000fa00d04180000080fa0000000600ca
:101318000000fa00c04180000080fa0000000600ca
:101328000200fa00000f78009e007800e1108800a3
:101338000080fa00000006000400fa001007980078
:101348009e009000010f78009e009000f00f200092
:10135800808f50000c0036001e4090000080fb007b
:101368000000400000407800e640600000cfb30075
:1013780000c07000104798001e4090000080fb00dd
:10138800d0108800030037001e4078000080fb0062
:10139800d01088001e007800e04188000080fa0024
:1013a800000006000200fa00000f78001e00780016
:1013b800e10f500009003200e10f5000030039002e
:1013c800e20f50000a003200150037003ec8bf0087
:1013d8000080fb00801088001100370010c0b300a7
:1013e8004de8b700c0842000bfff07000c0037009d
:1013f80080108000004078003ee8b700e1832000bc
:101408009140780040c6b30080cf500002003600fb
:10141800ccc2a90002003700ccc2a800000000001e
:1014280010c0b3000080fa00000006000000fa00b7
:101438000021ef00104e2e0010088800000328003d
:1014480020088800a04280000000e00002003a0066
:1014580060a62000200007008460a9009460a8000e
:101468005668ef000080fa00000006000200fa004b
:10147800000f78009e007800110888005668ef0079
:101488000080fa00000006000000fa001008800042
:101498000080fa00000006000200fa00000f780041
:1014a8009e007800010888005668ef000080fa0066
:1014b800000006000000fa00000880000080fa0022
:1014c800000006000000fa00cd02a900cce2a80046
:1014d8000080fa00000006000200fa00000f780001
:1014e8009460a9009e007800a14288009460a8003a
:1014f8000080fa00000006000000fa005668ef00bd
:101508009460a80005e1a8000080fa000000060029
:101518000000fa0005e1a9009460a9000080fa0023
:10152800000006000200fa00618520009140780062
:10153800014f78001e4078000004e00001003200ee
:101548005668ef001e4078000080fa000000060090
:101558000000fa0057c8bf000080fb000080fa00b6
:10156800000006000000fa005768ef000080fa004b
:10157800000006000000fa00890007003aff070093
:10158800c422a800201680000000d100614060003d
:101598000080fb0061006000211680000100a100ae
:1015a8000100700020168800c482a8002aff0700e6
:1015b8005ac8bf000080fb00b7fd07002aff0700dc
:1015c800ccc2a900cce2a800cd02a8006116800018
:1015d80000102000008060000000e00007003200da
:1015e8001dff070012c0b30051c0b300f0c0b30024
:1015f800b3fc07001cff0700f4ff370016ff0700c5
:101608000041eb0051c0b300f0c0b300acfc0700d0
:1016180015ff0700edff37000000fa000010230057
:10162800203a88004827ef004e27ef007027ef0088
:101638007227ef007427ef007627ef007a27ef0074
:101648007e27ef002200200080072000a10920004b
:1016580033742000804978008149780082497800f5
:101668000001eb00600420007105200023742000b5
:101678008049780081497800824978000080fa0022
:041688000000060058
:020000040000fa
:10168c003608000014000000000000004a080000aa
:10169c000a000000020000003001aa0001303100f5
:1016ac003233340000000000580800000200000033
:1016bc0002000000ffff00000008000020000000f6
:1016cc00000000005a0800000200000000000000aa
:1016dc002008000016000000000000005408000064
:0c16ec00040000000000000000000000ee
:020000040000fa
:1016f8000000fa00c422ef00cc22ef00400a2000cc
:1017080000168800f0432500401688005620ef0098
:101718005820ef006e20ef007020ef00c622ef0087
:10172800001c200070168800e024ef00000325004c
:10173800102788000080fa00000006000000fa0068
:10174800e1058000f0f82f00008060000040a00054
:10175800e005880021058000f0ff28000080600077
:1017680000c0a000200588000080fa0000000600e4
:101778000200fa00000f78009e007800c14288003d
:10178800ffff37000000fa00008020008007780083
:1017980080812000000188000080fa000000060017
:1017a8000000fa00d2ff07009bff0700e3ff0700d5
:1017b800b1fe070035fe07001cff07000080fa0095
:0417c8000000060017
:020000040000fa
:0200000401f009
:04000000ffffff00ff
:020000040000fa
:0200000401f009
:04000800ffffff00f7
:020000040000fa
:0200000401f009
:04000c005aff000097
:020000040000fa
:0200000401f009
:04001000baff000033
:020000040000fa
:0200000401f009
:040014005fff00008a
:020000040000fa
:0200000401f009
:04001800ffff0000e6
:020000040000fa
:0200000401f009
:04001c00ffff0000e2
:00000001FF
